:02000000082ACC
:08000800DF00030E8312B400B7
:0E0010000A0EB500040EB6008A110A122F2A3D
:1000200000000000D10B10280800CC08031D19287F
:100030000800F9300000000000000000000000008F
:1000400000000000000000000000000000000000B0
:1000500000000000FF3E031D1A2800000000000001
:100060000000000000000000000000000000000090
:10007000000000000000000000000000CC0B192868
:100080000800FA30CC001520FA30CC001520FA30E8
:10009000CC001520FA30CC001520CB0B41280800ED
:1000A0009F185028CD08031969281E08CE00CF01DB
:1000B000CE0DCF0DCE0DCF0DFC30CE0583161E0C10
:1000C0008312D000D00CD00E03305005CE04CF08E0
:1000D0006C281E08CE00CF0102301F049F004E087E
:1000E000D0004F08D100080007304E05D100510E56
:1000F000F03983169F0083124D08003A031D8928AA
:100100000130CA000030BA008530B90001308316D2
:1001100091008312390884000008C9004A08490484
:10012000D10080004D08D100D10DD10DFC3051051A
:1001300001389F004F0303191F175008D1001020EA
:1001400002301F049F000800831239088400490808
:1001500080008316910183129F01080010308312E2
:10016000CB008316071683124B08103A031D0800B4
:1001700010300705CB00B328FF308312CC00831664
:100180000716103083120705CC004C08CD0008007C
:10019000FF308312CC0083168716203083120705A8
:1001A000CC004C08CD0008008316051183120515FC
:1001B00008008316051183120511080083168711A4
:1001C0008312871108008316871183128715080090
:1001D000831607118312071508008316071183126F
:1001E00007110800831687108312871408008316EE
:1001F00087108312871008008316071083120714D4
:100200000800831607108312071008008312CD011F
:100210000330CE00CF012830D00074200130CD0053
:1002200050205008CB005108CC00A4204B08CD0032
:100230004C08CE0008008312CD010330CE00CF0160
:100240002830D0007420CD0150205008CB00A420CD
:100250004B08CC000800C820CB01CD08031D4B146F
:1002600044104B08031D4414441808000121D920F0
:100270006430CC001520F720E3206430CC0015203A
:10028000F220DE203829BC20CB01CD08031D4B1401
:1002900044114B08031D4415441D080001210A3078
:1002A000CC001520D920F720E3204416C411080003
:1002B000BC20CB01CD08031D4B1444114B08031D7A
:1002C000441544190800AE20D420DE20C7010A30AE
:1002D000470203187B29F220FF30CC001520F530AF
:1002E000CC001520F720FF30CC001520F530CC00D5
:1002F0001520C70A6729C415F2201B214C08C60027
:1003000046080A3C031898290121D920E820F22048
:10031000E320FF30CC0015202D30CC001520F72035
:10032000DE20FF30CC0015202D30CC001520862992
:10033000FC2044120800D9200121F720ED20E32001
:1003400008001B214C08C60046080A3C0318EA298D
:10035000450AC50045085A3C03180800C41C08009B
:10036000C5010121C8010A3048020318D32906211A
:100370004D08C60046080A3C0318C029450AC500B6
:10038000E820F220E320FF30CC0015202D30CC00F7
:100390001520F720DE20FF30CC0015202D30CC00BA
:1003A0001520C80AB32945080A3A031DE429D920B3
:1003B000E820F220E320C830CC001520F720DE2012
:1003C000C830CC001520D929C501FC20ED20F22031
:1003D000DE200800C5010800831691010730831252
:1003E0009900C0308316810001308312CB00412078
:1003F00044164410C6014411C411C501C4149B2104
:10040000441A5821C41D002A2B21A1214321002A6E
:10041000D5308312A000C430A100BB30A200DC3074
:10042000A300A401A501A601A701A801A901AA0191
:10043000AB01AC01AD01AE01AF01BE01BF01B7011F
:10044000B801C001C101C201C301B001B101B201D3
:10045000B301BC01BD01BB018A110A12EC29831250
:10046000360E8400350E8A00340E8300DF0E5F0ED8
:02047000090081
:02400E00420E60
:00000001FF
